:020000040000FA
:04080000A6EF06F069
:1008100003B207EF05F0F2B422EF05F09EB02AEF25
:1008200005F09EB232EF05F0F2A81AEF04F0F2B232
:100830001CEF04F084EF06F0CD90F2929EA026EF1C
:1008400004F00101533F26EF04F0542BAEC1B2F186
:10085000AFC1B3F1B0C1B4F1B1C1B5F1AAC1AEF14C
:10086000ABC1AFF1ACC1B0F1ADC1B1F1A6C1AAF15C
:10087000A7C1ABF1A8C1ACF1A9C1ADF1A2C1A6F16C
:10088000A3C1A7F1A4C1A8F1A5C1A9F19EC1A2F17C
:100890009FC1A3F1A0C1A4F1A1C1A5F19AC19EF18C
:1008A0009BC19FF19CC1A0F19DC1A1F196C19AF19C
:1008B00097C19BF198C19CF199C19DF1CECF96F162
:1008C000CFCF97F153C198F154C199F1CF6ACE6A55
:1008D0000101536B546B9E90CD800EBC0E8E0EBAF0
:1008E00075EF04F00E8A84EF06F00E8C0EBEB1EFA9
:1008F00004F096C19AF197C19BF198C19CF199C1FE
:100900009DF19AC19EF19BC19FF19CC1A0F19DC137
:10091000A1F19EC1A2F19FC1A3F1A0C1A4F1A1C107
:10092000A5F1A2C1A6F1A3C1A7F1A4C1A8F1A5C1D7
:10093000A9F1A6C1AAF1A7C1ABF1A8C1ACF1A9C1A7
:10094000ADF1AAC1AEF1ABC1AFF1ACC1B0F1ADC177
:10095000B1F1AEC1B2F1AFC1B3F1B0C1B4F1B1C147
:10096000B5F101015E6B5F6B606B616B96515E2749
:1009700097515F2398516023995161239A515E27C3
:100980009B515F239C5160239D5161239E515E27A3
:100990009F515F23A0516023A1516123A2515E2783
:1009A000A3515F23A4516023A5516123A6515E2763
:1009B000A7515F23A8516023A9516123AA515E2743
:1009C000AB515F23AC516023AD516123AE515E2723
:1009D000AF515F23B0516023B1516123B2515E2703
:1009E000B3515F23B4516023B5516123D890613373
:1009F00060335F335E33D890613360335F335E338F
:100A0000D890613360335F335E3384EF06F0039236
:100A1000030103EE00F080517F0BE92604C0EFFFD5
:100A2000802B8151805D700BD8A48B820000805197
:100A3000815D700BD8A48B9281518019D8B4079036
:100A400084EF06F0F2940101453F84EF06F0462B57
:100A500084EF06F09E900101533F84EF06F0542B83
:100A600084EF06F09E92C3CF55F1C4CF56F1C282F7
:100A700007B49DEF05F047C14BF148C14CF149C1A6
:100A80004DF14AC14EF15EC162F15FC163F160C1D7
:100A900064F161C165F196C1B6F197C1B7F198C132
:100AA000B8F199C1B9F19AC1BAF19BC1BBF19CC12E
:100AB000BCF19DC1BDF19EC1BEF19FC1BFF1A0C1FE
:100AC000C0F1A1C1C1F1A2C1C2F1A3C1C3F1A4C1CE
:100AD000C4F1A5C1C5F1A6C1C6F1A7C1C7F1A8C19E
:100AE000C8F1A9C1C9F1AAC1CAF1ABC1CBF1ACC16E
:100AF000CCF1ADC1CDF1AEC1CEF1AFC1CFF1B0C13E
:100B0000D0F1B1C1D1F1B2C1D2F1B3C1D3F1B4C10D
:100B1000D4F1B5C1D5F1010155515B2756515C2384
:100B2000E86A5D230D2E9DEF05F05CC157F15DC1B4
:100B300058F15B6B5C6B5D6B078E0201002F84EFDD
:100B400006F03C0E006F00C10CF101C10DF102C1B5
:100B50000EF103C10FF104C110F105C111F106C17D
:100B600012F107C113F108C114F109C115F10AC14D
:100B700016F10BC117F134C135F101018A67C8EFD5
:100B800005F08B67C8EF05F08C67C8EF05F08D673F
:100B9000CCEF05F0FCEF05F08EC100F18FC101F143
:100BA00090C102F191C103F10101010E046F000E29
:100BB000056F000E066F000E076F98EC14F000C171
:100BC0008EF101C18FF102C190F103C191F1006773
:100BD000F1EF05F00167F1EF05F00267F1EF05F0C5
:100BE0000367FCEF05F08AC18EF18BC18FF18CC1D8
:100BF00090F18DC191F10E80D57ED5BE69D0D6CF52
:100C000047F1D7CF48F145C149F1E86AE8CF4AF149
:100C10000F9047C100F148C101F149C102F14AC139
:100C200003F101010A0E046F000E056F000E066F3E
:100C3000000E076F98EC14F000AF0F80010154A76D
:100C40002EEF06F00E9A0E9C0E9E0101000E5E6FB6
:100C5000600E5F6F3D0E606F080E616F010147BF50
:100C60003EEF06F048673EEF06F049673EEF06F0BC
:100C70004A673EEF06F0F28863EF06F0F2985E6B8B
:100C80005F6B606B616B966B976B986B996B9A6BF4
:100C90009B6B9C6B9D6B9E6B9F6BA06BA16BA26B08
:100CA000A36BA46BA56BA66BA76BA86BA96BAA6BB8
:100CB000AB6BAC6BAD6BAE6BAF6BB06BB16BB26B68
:100CC000B36BB46BB56BD76AD66A0101456B466BE3
:100CD0000CC100F10DC101F10EC102F10FC103F110
:100CE00010C104F111C105F112C106F113C107F1E0
:100CF00014C108F115C109F116C10AF117C10BF1B0
:100D000035C134F184EF06F002C0E0FF005001C0AD
:100D1000D8FF1000A6B28AEF06F00CC0A9FF0BC0E6
:100D2000A8FFA69EA69CA684F29E550EA76EAA0EAC
:100D3000A76EA682F28EA694A6B29CEF06F01200D1
:100D4000A96EA69EA69CA680A8501200076A0E6AED
:100D50000F6A0F010E0EC16E860EC06E030EC26EBC
:100D60000F01896A190E926E080E8A6EF10E936E4B
:100D70008B6A800E946EF18E0D6A01015B6B5C6B69
:100D80005D6B576B586BF29A0101476B486B496B6F
:100D90004A6B4B6B4C6B4D6B4E6B4F6B506B516B8F
:100DA000526B456B466BD76AD66A0F01280ED56E1B
:100DB000F28A9D90B00ECD6E01015E6B5F6B606B31
:100DC000616B626B636B646B656B666B676B686BA7
:100DD000696B536B546BCF6ACE6A0E9A0E9C0E9E53
:100DE0009D80760ECA6E9D8202013C0E006FCC6A19
:100DF000160EA0EC06F0E8CF00F1170EA0EC06F0FE
:100E0000E8CF01F1180EA0EC06F0E8CF02F1190EC0
:100E1000A0EC06F0E8CF03F1010103AF2AEF07F0E1
:100E20008FEC15F0160E0C6E00C10BF08AEC06F07C
:100E3000170E0C6E01C10BF08AEC06F0180E0C6E4A
:100E400002C10BF08AEC06F0190E0C6E03C10BF018
:100E50008AEC06F000C18AF101C18BF102C18CF16C
:100E600003C18DF100C18EF101C18FF102C190F17A
:100E700003C191F11A0EA0EC06F0E8CF00F11B0EB1
:100E8000A0EC06F0E8CF01F11C0EA0EC06F0E8CFD4
:100E900002F11D0EA0EC06F0E8CF03F1010103AF53
:100EA00080EF07F08FEC15F01A0E0C6E00C10BF0FE
:100EB0008AEC06F01B0E0C6E01C10BF08AEC06F0FA
:100EC0001C0E0C6E02C10BF08AEC06F01D0E0C6EAF
:100ED00003C10BF08AEC06F01A0EA0EC06F0E8CF86
:100EE00000F11B0EA0EC06F0E8CF01F11C0EA0EC07
:100EF00006F0E8CF02F11D0EA0EC06F0E8CF03F1FA
:100F000000C192F101C193F102C194F103C195F1C5
:100F1000240EAC6E900EAB6E240EAC6E080EB86E46
:100F200080B6B1EF07F01E0EA0EC06F0E8CF00F19E
:100F30001F0EA0EC06F0E8CF01F100C1E8FFFF0AA8
:100F400010E001C1E8FFFF0A0CE01E0EA0EC06F065
:100F5000E8CFAFFF1F0EA0EC06F0E8CFB0FFB5EF73
:100F600007F0010EB06E7F0EAF6E0401806B816BD7
:100F70000F01900EAB6E0F019D8A0301806B816B98
:100F8000A26B8B9207900001F28EF28C07B05FEF9C
:100F900012F00EB040EF0DF00301805181197F0B6C
:100FA000D8B45FEF12F013EE00F081517F0BE12611
:100FB000812BE7CFE8FFE00BD8B45FEF12F023EE10
:100FC00082F0A2511F0BD926E7CFDFFFA22BDF5003
:100FD000780AD8A45FEF12F007808EC100F18FC1AC
:100FE00001F190C102F191C103F10101040E046FFE
:100FF000000E056F000E066F000E076F98EC14F0E0
:1010000000AF0CEF08F00101030E8E6F000E8F6F22
:10101000000E906F000E916F03018251720AD8B4D6
:1010200040EF0DF08251520AD8B440EF0DF08251DA
:10103000750AD8B440EF0DF08251630AD8B41BEFA3
:101040000FF08251690AD8B4FEEF09F082517A0A92
:10105000D8B411EF0BF08251490AD8B49DEF09F0D2
:101060008251500AD8B4BBEF08F08251700AD8B44C
:10107000FEEF08F08251540AD8B429EF09F08251EA
:10108000740AD8B46FEF09F08251730AD8B470EFC4
:101090000CF08251530AD8B4D5EF0CF08251620A99
:1010A000D8B46DEF08F08251420AD8B4A8EF08F026
:1010B00050EF0FF0040114EE00F080517F0BE12699
:1010C00082C4E7FF802B12000D0E826F5AEC08F0ED
:1010D0000A0E826F5AEC08F012008351610AD8A4FC
:1010E00050EF0FF08451750AD8A450EF0FF08551DE
:1010F000640AD8A450EF0FF086C32AF187C32BF1FE
:1011000088C32CF189C32DF18AC32EF18BC32FF133
:101110008CC330F18DC331F18EC332F18FC333F103
:101120000101296BDDEC15F054EC15F000C1AFFFA7
:1011300001C1B0FF1E0E0C6EAFCF0BF08AEC06F0B3
:101140001F0E0C6EB0CF0BF08AEC06F050EF0FF0D4
:1011500080B6B2EF08F00401300E826F5AEC08F04E
:10116000B7EF08F00401310E826F5AEC08F064EC1E
:1011700008F050EF0FF083C32AF184C32BF185C32D
:101180002CF186C32DF187C32EF188C32FF189C3BB
:1011900030F18AC331F18BC332F18CC333F10101D9
:1011A000DDEC15F054EC15F0160E0C6E00C10BF0D2
:1011B0008AEC06F0170E0C6E01C10BF08AEC06F0FB
:1011C000180E0C6E02C10BF08AEC06F0190E0C6EB4
:1011D00003C10BF08AEC06F000C18AF101C18BF16A
:1011E00002C18CF103C18DF100C18EF101C18FF1FB
:1011F00002C190F103C191F19DEF09F083C32AF17F
:1012000084C32BF185C32CF186C32DF187C32EF146
:1012100088C32FF189C330F18AC331F18BC332F116
:101220008CC333F10101DDEC15F054EC15F000C175
:101230008AF101C18BF102C18CF103C18DF100C1B2
:101240008EF101C18FF102C190F103C191F19DEFC7
:1012500009F083C32AF184C32BF185C32CF186C323
:101260002DF187C32EF188C32FF189C330F18AC3D2
:1012700031F18CC332F18DC333F10101DDEC15F096
:1012800054EC15F00101000E046F000E056F010E05
:10129000066F000E076FA7EC14F01A0E0C6E00C15B
:1012A0000BF08AEC06F01B0E0C6E01C10BF08AEC01
:1012B00006F01C0E0C6E02C10BF08AEC06F01D0E3F
:1012C0000C6E03C10BF08AEC06F000C192F101C173
:1012D00093F102C194F103C195F19DEF09F083C32D
:1012E0002AF184C32BF185C32CF186C32DF187C36A
:1012F0002EF188C32FF189C330F18AC331F18CC339
:1013000032F18DC333F10101DDEC15F054EC15F031
:101310000101000E046F000E056F010E066F000E36
:10132000076FA7EC14F000C192F101C193F102C163
:1013300094F103C195F19DEF09F0160EA0EC06F0B3
:10134000E8CF00F1170EA0EC06F0E8CF01F1180E7F
:10135000A0EC06F0E8CF02F1190EA0EC06F0E8CF01
:1013600003F132EC15F05EEC13F00401730E826FA2
:101370005AEC08F004012C0E826F5AEC08F08AC176
:1013800000F18BC101F18CC102F18DC103F132EC8E
:1013900015F05EEC13F00401730E826F5AEC08F046
:1013A00004012C0E826F5AEC08F01A0EA0EC06F025
:1013B000E8CF00F11B0EA0EC06F0E8CF01F11C0E07
:1013C000A0EC06F0E8CF02F11D0EA0EC06F0E8CF8D
:1013D00003F16BEC0FF004012C0E826F5AEC08F055
:1013E00092C100F193C101F194C102F195C103F1E1
:1013F0006BEC0FF064EC08F050EF0FF00401690E95
:10140000826F5AEC08F004012C0E826F5AEC08F03F
:101410000101040E006F000E016F000E026F000E3E
:10142000036F32EC15F02CC182F40401300E8227D8
:101430005AEC08F02DC182F40401300E82275AECD8
:1014400008F02EC182F40401300E82275AEC08F015
:101450002FC182F40401300E82275AEC08F030C10B
:1014600082F40401300E82275AEC08F031C182F474
:101470000401300E82275AEC08F032C182F40401D4
:10148000300E82275AEC08F033C182F40401300E8A
:1014900082275AEC08F004012C0E826F5AEC08F0F7
:1014A0000101050E006F000E016F000E026F000EAD
:1014B000036F32EC15F02CC182F40401300E822748
:1014C0005AEC08F02DC182F40401300E82275AEC48
:1014D00008F02EC182F40401300E82275AEC08F085
:1014E0002FC182F40401300E82275AEC08F030C17B
:1014F00082F40401300E82275AEC08F031C182F4E4
:101500000401300E82275AEC08F032C182F4040143
:10151000300E82275AEC08F033C182F40401300EF9
:1015200082275AEC08F004012C0E826F5AEC08F066
:101530000101190E006F000E016F000E026F000E08
:10154000036F32EC15F02CC182F40401300E8227B7
:101550005AEC08F02DC182F40401300E82275AECB7
:1015600008F02EC182F40401300E82275AEC08F0F4
:101570002FC182F40401300E82275AEC08F030C1EA
:1015800082F40401300E82275AEC08F031C182F453
:101590000401300E82275AEC08F032C182F40401B3
:1015A000300E82275AEC08F033C182F40401300E69
:1015B00082275AEC08F004012C0E826F5AEC08F0D6
:1015C000200EF86EF76AF66A04010900F5CF82F47E
:1015D0005AEC08F00900F5CF82F45AEC08F0090043
:1015E000F5CF82F45AEC08F00900F5CF82F45AECFA
:1015F00008F00900F5CF82F45AEC08F00900F5CFA5
:1016000082F45AEC08F00900F5CF82F45AEC08F0A5
:101610000900F5CF82F45AEC08F064EC08F050EFC2
:101620000FF08351630AD8A450EF0FF08451610A80
:10163000D8A450EF0FF085516C0AD8A450EF0FF0EA
:101640008651410A3FE08651440A1BE08651420A16
:10165000D8B475EF0BF08651350AD8B4DAEF10F034
:101660008651360AD8B42FEF11F08651370AD8B414
:1016700098EF11F08651380AD8B4F6EF11F050EF18
:101680000FF00798079A04017A0E826F5AEC08F05F
:101690000401780E826F5AEC08F00401640E826F28
:1016A0005AEC08F00401550E826F5AEC08F05EEF18
:1016B0000BF004014C0E826F5AEC08F064EC08F059
:1016C00050EF0FF00788079A04017A0E826F5AECE8
:1016D00008F00401410E826F5AEC08F00401610E1B
:1016E000826F5AEC08F052EF0BF00798078A04015A
:1016F0007A0E826F5AEC08F00401420E826F5AECA7
:1017000008F00401610E826F5AEC08F052EF0BF002
:101710000101666793EF0BF0676793EF0BF0686763
:1017200093EF0BF06967ABEF0BF04F679FEF0BF098
:1017300050679FEF0BF051679FEF0BF05267ABEFD5
:101740000BF00101000E006F000E016F000E026F22
:10175000000E036F12000101620E046F010E056F8F
:10176000000E066F000E076F66C100F167C101F140
:1017700068C102F169C103F198EC14F003BF2FEFC7
:101780000CF00101000E046FA80E056F550E066FD8
:10179000020E076F66C100F167C101F168C102F175
:1017A00069C103F166C186F167C187F168C188F13B
:1017B00069C189F198EC14F003BFE8EF0BF0010167
:1017C000000E866FA80E876F550E886F020E896F08
:1017D0000E0EA0EC06F0E8CF18F10F0EA0EC06F00C
:1017E000E8CF19F1100EA0EC06F0E8CF1AF1110EB7
:1017F000A0EC06F0E8CF1BF1E1EC13F086C104F198
:1018000087C105F188C106F189C107F198EC14F090
:101810000782A5EC13F0E1EC13F00792A5EC13F0AE
:1018200086C100F187C101F188C102F189C103F1CC
:101830000792A5EC13F0CC0E046FE00E056F870E37
:10184000066F050E076F98EC14F000C118F101C186
:1018500019F102C11AF103C11BF167EF0CF001018C
:10186000800E006F1A0E016F060E026F000E036FDE
:101870004FC104F150C105F151C106F152C107F148
:1018800098EC14F003AF48EF0CF08FEC15F0120059
:101890000E0EA0EC06F0E8CF18F10F0EA0EC06F04B
:1018A000E8CF19F1100EA0EC06F0E8CF1AF1110EF6
:1018B000A0EC06F0E8CF1BF14FC100F150C101F1DF
:1018C00051C102F152C103F10782A5EC13F018C116
:1018D00000F119C101F11AC102F11BC103F112009B
:1018E0000401730E826F5AEC08F004012C0E826F13
:1018F0005AEC08F0078462C166F163C167F164C104
:1019000068F165C169F14BC14FF14CC150F14DC156
:1019100051F14EC152F157C159F158C15AF10794D2
:1019200096EC0CF064EC08F050EF0FF066C100F19B
:1019300067C101F168C102F169C103F1010132EC33
:1019400015F05EEC13F00401630E826F5AEC08F0A0
:1019500004012C0E826F5AEC08F04FC100F150C107
:1019600001F151C102F152C103F1010132EC15F054
:101970005EEC13F00401660E826F5AEC08F004016D
:101980002C0E826F5AEC08F08FEC15F059C100F163
:101990005AC101F1010132EC15F05EEC13F00401C3
:1019A000740E826F5AEC08F012000F820401530E7D
:1019B000826F5AEC08F004012C0E826F5AEC08F08A
:1019C00083C32AF184C32BF185C32CF186C32DF187
:1019D00087C32EF188C32FF189C330F18AC331F157
:1019E0008BC332F18CC333F10101DDEC15F054EC03
:1019F00015F000C166F101C167F102C168F103C1D0
:101A000069F18EC32AF18FC32BF190C32CF191C3DE
:101A10002DF192C32EF193C32FF194C330F195C3EE
:101A200031F196C332F197C333F10101DDEC15F0CA
:101A300054EC15F000C14FF101C150F102C151F158
:101A400003C152F1D0EC15F099C32FF19AC330F1D4
:101A50009BC331F19CC332F19DC333F10101DDEC35
:101A600015F054EC15F000C159F101C15AF196EC92
:101A70000CF004012C0E826F5AEC08F047EF0DF0C9
:101A80008251520A03E10E8247EF0DF00E9282510D
:101A9000750A03E10F844EEF0DF00F948251550A41
:101AA00003E10F8655EF0DF00F9607840FB2B2EFEA
:101AB0000DF00FA49EEF0DF0B6C166F1B7C167F14E
:101AC000B8C168F1B9C169F1BAC16AF1BBC16BF1C2
:101AD000BCC16CF1BDC16DF1BEC16EF1BFC16FF192
:101AE000C0C170F1C1C171F1C2C172F1C3C173F162
:101AF000C4C174F1C5C175F1C6C176F1C7C177F132
:101B0000C8C178F1C9C179F1CAC17AF1CBC17BF101
:101B1000CCC17CF1CDC17DF1CEC17EF1CFC17FF1D1
:101B2000D0C180F1D1C181F1D2C182F1D3C183F1A1
:101B3000D4C184F1D5C185F1A6EF0DF062C166F183
:101B400063C167F164C168F165C169F14BC14FF1CF
:101B50004CC150F14DC151F14EC152F157C159F133
:101B600058C15AF107940EA0D4EF0DF0010192670D
:101B7000C1EF0DF09367C1EF0DF09467C1EF0DF069
:101B80009567C5EF0DF0D4EF0DF088EC0BF092C126
:101B900004F193C105F194C106F195C107F198ECE8
:101BA00014F003BF18EF0FF088EC0BF00101000EEA
:101BB000046F000E056F010E066F000E076FC6EC76
:101BC00014F00FA4EBEF0DF00401750E826F5AECC8
:101BD00008F0F0EF0DF00401720E826F5AEC08F07D
:101BE00004012C0E826F5AEC08F032EC15F02967D4
:101BF000FFEF0DF00401200E826F02EF0EF00401E2
:101C00002D0E826F5AEC08F030C182F40401300EC0
:101C100082275AEC08F031C182F40401300E822789
:101C20005AEC08F004012E0E826F5AEC08F032C113
:101C300082F40401300E82275AEC08F033C182F49A
:101C40000401300E82275AEC08F004016D0E826FF9
:101C50005AEC08F004012C0E826F5AEC08F04FC1C8
:101C600000F150C101F151C102F152C103F1010172
:101C700032EC15F05EEC13F00401480E826F5AEC62
:101C800008F004017A0E826F5AEC08F004012C0E61
:101C9000826F5AEC08F066C100F167C101F168C1BA
:101CA00002F169C103F1010132EC15F05EEC13F0B1
:101CB0000401630E826F5AEC08F004012C0E826F4F
:101CC0005AEC08F066C100F167C101F168C102F188
:101CD00069C103F101010A0E046F000E056F000EC9
:101CE000066F000E076FA7EC14F0000E046F120EC3
:101CF000056F000E066F000E076FC6EC14F032EC95
:101D000015F02AC182F40401300E82275AEC08F043
:101D10002BC182F40401300E82275AEC08F02CC14A
:101D200082F40401300E82275AEC08F02DC182F4AF
:101D30000401300E82275AEC08F02EC182F404010F
:101D4000300E82275AEC08F02FC182F40401300EC5
:101D500082275AEC08F030C182F40401300E822749
:101D60005AEC08F004012E0E826F5AEC08F031C1D3
:101D700082F40401300E82275AEC08F032C182F45A
:101D80000401300E82275AEC08F033C182F40401BA
:101D9000300E82275AEC08F00401730E826F5AEC61
:101DA00008F004012C0E826F5AEC08F08FEC15F04D
:101DB00059C100F15AC101F17AEC10F00EB2E4EF12
:101DC0000EF00EA016EF0FF004012C0E826F5AECED
:101DD00008F0200EF86EF76AF66A04010900F5CFE4
:101DE00082F45AEC08F00900F5CF82F45AEC08F0BE
:101DF0000900F5CF82F45AEC08F00900F5CF82F41F
:101E00005AEC08F00900F5CF82F45AEC08F009000A
:101E1000F5CF82F45AEC08F00900F5CF82F45AECC1
:101E200008F00900F5CF82F45AEC08F064EC08F0F1
:101E30000E9050EF0FF00401630E826F5AEC08F021
:101E400004012C0E826F5AEC08F056EC0FF00401DE
:101E50002C0E826F5AEC08F0C9EC0FF004012C0E26
:101E6000826F5AEC08F045EC10F004012C0E826FE2
:101E70005AEC08F00101F80E006FCD0E016F660EEE
:101E8000026F030E036F6BEC0FF004012C0E826FD8
:101E90005AEC08F05BEC10F064EC08F050EF0FF037
:101EA0000301A26B07900F925FEF12F0D8900E0E15
:101EB000A0EC06F0E8CF00F10F0EA0EC06F0E8CFA2
:101EC00001F1100EA0EC06F0E8CF02F1110EA0EC2B
:101ED00006F0E8CF03F10101000E046F000E056F5C
:101EE000010E066F000E076FC6EC14F032EC15F011
:101EF0002AC182F40401300E82275AEC08F02BC16B
:101F000082F40401300E82275AEC08F02CC182F4CE
:101F10000401300E82275AEC08F02DC182F404012E
:101F2000300E82275AEC08F02EC182F40401300EE4
:101F300082275AEC08F02FC182F40401300E822768
:101F40005AEC08F030C182F40401300E82275AECBA
:101F500008F031C182F40401300E82275AEC08F0F7
:101F600004012E0E826F5AEC08F032C182F4040193
:101F7000300E82275AEC08F033C182F40401300E8F
:101F800082275AEC08F004016D0E826F5AEC08F0BB
:101F90001200120EA0EC06F0E8CF00F1130EA0EC38
:101FA00006F0E8CF01F1140EA0EC06F0E8CF02F144
:101FB000150EA0EC06F0E8CF03F101010A0E046F44
:101FC000000E056F000E066F000E076FA7EC14F0F1
:101FD000000E046F120E056F000E066F000E076FE5
:101FE000C6EC14F032EC15F02AC182F40401300E74
:101FF00082275AEC08F02BC182F40401300E8227AC
:102000005AEC08F02CC182F40401300E82275AECFD
:1020100008F02DC182F40401300E82275AEC08F03A
:102020002EC182F40401300E82275AEC08F02FC131
:1020300082F40401300E82275AEC08F030C182F499
:102040000401300E82275AEC08F004012E0E826F34
:102050005AEC08F031C182F40401300E82275AECA8
:1020600008F032C182F40401300E82275AEC08F0E5
:1020700033C182F40401300E82275AEC08F00401C7
:10208000730E826F5AEC08F012000A0EA0EC06F0F4
:10209000E8CF00F10B0EA0EC06F0E8CF01F10C0E3A
:1020A000A0EC06F0E8CF02F10D0EA0EC06F0E8CFB0
:1020B00003F17AEF10F0060EA0EC06F0E8CF00F185
:1020C000070EA0EC06F0E8CF01F1080EA0EC06F038
:1020D000E8CF02F1090EA0EC06F0E8CF03F17AEFA9
:1020E00010F001018FEC15F0078457C100F158C1C1
:1020F00001F107940101E80E046F800E056F000ED8
:10210000066F000E076FA7EC14F0000E046F040EAC
:10211000056F000E066F000E076FC6EC14F0880EF8
:10212000046F130E056F000E066F000E076F98EC1C
:1021300014F00A0E046F000E056F000E066F000EFD
:10214000076FC6EC14F032EC15F001012967AEEF11
:1021500010F00401200E826FB1EF10F004012D0E7B
:10216000826F5AEC08F030C182F40401300E8227ED
:102170005AEC08F031C182F40401300E82275AEC87
:1021800008F032C182F40401300E82275AEC08F0C4
:1021900004012E0E826F5AEC08F033C182F4040160
:1021A000300E82275AEC08F00401430E826F5AEC7D
:1021B00008F0120087C32AF188C32BF189C32CF1E0
:1021C0008AC32DF18BC32EF18CC32FF18DC330F157
:1021D0008EC331F190C332F191C333F10101296B08
:1021E000DDEC15F054EC15F00101000E046F000E4B
:1021F000056F010E066F000E076FA7EC14F00E0EB0
:102200000C6E00C10BF08AEC06F00F0E0C6E01C1D3
:102210000BF08AEC06F0100E0C6E02C10BF08AEC8B
:1022200006F0110E0C6E03C10BF08AEC06F00401EF
:102230007A0E826F5AEC08F004012C0E826F5AEC71
:1022400008F00401350E826F5AEC08F004012C0EE0
:10225000826F5AEC08F056EC0FF05EEF0BF087C37C
:102260002AF188C32BF189C32CF18AC32DF18BC3CA
:102270002EF18CC32FF18DC330F18EC331F190C399
:1022800032F191C333F10101296BDDEC15F054EC0F
:1022900015F0880E046F130E056F000E066F000E0A
:1022A000076F9CEC14F0000E046F040E056F000E17
:1022B000066F000E076FA7EC14F00101E80E046F23
:1022C000800E056F000E066F000E076FC6EC14F04F
:1022D0000A0E0C6E00C10BF08AEC06F00B0E0C6EB1
:1022E00001C10BF08AEC06F00C0E0C6E02C10BF073
:1022F0008AEC06F00D0E0C6E03C10BF08AEC06F0B2
:1023000004017A0E826F5AEC08F004012C0E826FE1
:102310005AEC08F00401360E826F5AEC08F0040102
:102320002C0E826F5AEC08F045EC10F05EEF0BF0CB
:1023300087C32AF188C32BF189C32CF18AC32DF1FD
:102340008BC32EF18CC32FF18DC330F18FC331F1CC
:1023500090C332F191C333F10101DDEC15F054EC7F
:1023600015F0000E046F120E056F000E066F000EC2
:10237000076FA7EC14F001010A0E046F000E056F41
:10238000000E066F000E076FC6EC14F0120E0C6EF6
:1023900000C10BF08AEC06F0130E0C6E01C10BF0BD
:1023A0008AEC06F0140E0C6E02C10BF08AEC06F0FB
:1023B000150E0C6E03C10BF08AEC06F004017A0EC8
:1023C000826F5AEC08F004012C0E826F5AEC08F070
:1023D0000401370E826F5AEC08F004012C0E826F54
:1023E0005AEC08F0C9EC0FF05EEF0BF087C32AF14E
:1023F00088C32BF189C32CF18AC32DF18BC32EF135
:102400008CC32FF18DC330F18EC331F190C332F103
:1024100091C333F10101296BDDEC15F054EC15F09B
:10242000880E046F130E056F000E066F000E076F07
:102430009CEC14F0000E046F040E056F000E066F86
:10244000000E076FA7EC14F00101E80E046F800E78
:10245000056F000E066F000E076FC6EC14F0060E37
:102460000C6E00C10BF08AEC06F0070E0C6E01C179
:102470000BF08AEC06F0080E0C6E02C10BF08AEC31
:1024800006F0090E0C6E03C10BF08AEC06F0040195
:102490007A0E826F5AEC08F004012C0E826F5AEC0F
:1024A00008F00401380E826F5AEC08F004012C0E7B
:1024B000826F5AEC08F05BEC10F05EEF0BF007A8AF
:1024C000D3EF12F00101800E006F1A0E016F060E9D
:1024D000026F000E036F4BC104F14CC105F14DC1F9
:1024E00006F14EC107F198EC14F003BF1AEF13F098
:1024F00058EC13F04BC100F14CC101F14DC102F198
:102500004EC103F10782A5EC13F018C104F119C103
:1025100005F11AC106F11BC107F1F80E006FCD0ECF
:10252000016F660E026F030E036F98EC14F00E0E2F
:102530000C6E00C10BF08AEC06F00F0E0C6E01C1A0
:102540000BF08AEC06F0100E0C6E02C10BF08AEC58
:1025500006F0110E0C6E03C10BF08AEC06F0078436
:1025600001018FEC15F057C100F158C101F107943A
:102570000A0E0C6E00C10BF08AEC06F00B0E0C6E0E
:1025800001C10BF08AEC06F00C0E0C6E02C10BF0D0
:102590008AEC06F00D0E0C6E03C10BF08AEC06F00F
:1025A00007981AEF13F007AA1AEF13F00784010136
:1025B0008FEC15F057C100F158C101F10794060ED8
:1025C0000C6E00C10BF08AEC06F0070E0C6E01C118
:1025D0000BF08AEC06F0080E0C6E02C10BF08AECD0
:1025E00006F0090E0C6E03C10BF08AEC06F00784AE
:1025F00062C100F163C101F164C102F165C103F17F
:102600000794120E0C6E00C10BF08AEC06F0130E4C
:102610000C6E01C10BF08AEC06F0140E0C6E02C1B8
:102620000BF08AEC06F0150E0C6E03C10BF08AEC71
:1026300006F0079A0401805181197F0B0BE09EA8D8
:1026400009D014EE00F081517F0BE126E750812B79
:102650000F01AD6EC6EF07F018C100F119C101F10D
:102660001AC102F11BC103F1000E046F000E056FC9
:10267000010E066F000E076FC6EC14F029A157EF8C
:1026800013F02051D8B457EF13F018C100F119C15D
:1026900001F11AC102F11BC103F1000E046F000E1B
:1026A000056F0A0E066F000E076FC6EC14F01200DD
:1026B0000101186B196B1A6B1B6B12002AC182F493
:1026C0000401300E82275AEC08F02BC182F4040179
:1026D000300E82275AEC08F02CC182F40401300E2F
:1026E00082275AEC08F02DC182F40401300E8227B3
:1026F0005AEC08F02EC182F40401300E82275AEC05
:1027000008F02FC182F40401300E82275AEC08F041
:1027100030C182F40401300E82275AEC08F031C136
:1027200082F40401300E82275AEC08F032C182F4A0
:102730000401300E82275AEC08F033C182F4040100
:10274000300E82275AEC08F012000101005305E117
:10275000015303E1025301E1002B68EC14F08FEC0C
:1027600015F03951006F3A51016F420E046F4B0E54
:10277000056F000E066F000E076FA7EC14F000C186
:1027800004F101C105F102C106F103C107F118C14D
:1027900000F119C101F11AC102F11BC103F107B225
:1027A000D6EF13F09CEC14F0D8EF13F098EC14F083
:1027B00000C118F101C119F102C11AF103C11BF1E5
:1027C00012008FEC15F059C100F15AC101F1060E4B
:1027D000A0EC06F0E8CF04F1070EA0EC06F0E8CF7D
:1027E00005F1080EA0EC06F0E8CF06F1090EA0EC0A
:1027F00006F0E8CF07F198EC14F000C124F101C114
:1028000025F102C126F103C127F1290E046F000E44
:10281000056F000E066F000E076FA7EC14F0EE0EAA
:10282000046F430E056F000E066F000E076F9CECE1
:1028300014F024C104F125C105F126C106F127C118
:1028400007F1A7EC14F000C11CF101C11DF102C198
:102850001EF103C11FF1120EA0EC06F0E8CF04F147
:10286000130EA0EC06F0E8CF05F1140EA0EC06F074
:10287000E8CF06F1150EA0EC06F0E8CF07F10D0E3B
:10288000006F000E016F000E026F000E036FA7ECC9
:1028900014F0180E046F000E056F000E066F000E88
:1028A000076FC6EC14F01CC104F11DC105F11EC177
:1028B00006F11FC107F19CEC14F06A0E046F2A0E9A
:1028C000056F000E066F000E076F98EC14F01200F3
:1028D000BF0EFA6E200E3A6F396BD8900037013771
:1028E00002370337D8B079EF14F03A2F6EEF14F0B7
:1028F00039073A070353D8B412000331070B800994
:102900003F6F03390F0B010F396F80EC5FF0406FA1
:10291000390580EC5FF0405D405F396B3F33D8B0E4
:10292000392739333FA98EEF14F04051392712006F
:10293000B4EC15F0D8B0120003510719346F77ECDE
:1029400015F0D8900751031934AF800F1200346B83
:102950009BEC15F0D8A0B1EC15F0D8B0120086ECC5
:1029600015F08FEC15F01F0E366FC7EC15F00B3518
:10297000D8B077EC15F0D8A00335D8B01200362FB8
:10298000B5EF14F034B19EEC15F01200346B045125
:102990000511061107110008D8A09BEC15F0D8A06E
:1029A000B1EC15F0D8B01200086B096B0A6B0B6B19
:1029B000C7EC15F01F0E366FC7EC15F007510B5D15
:1029C000D8A4EFEF14F006510A5DD8A4EFEF14F08D
:1029D0000551095DD8A4EFEF14F00451085DD8A0AB
:1029E00002EF15F00451085F0551D8A0053D095FBD
:1029F0000651D8A0063D0A5F0751D8A0073D0B5FDE
:102A0000D8900081362FDCEF14F034B19EEC15F035
:102A1000346B9BEC15F0D890CBEC15F007510B5DA7
:102A2000D8A41FEF15F006510A5DD8A41FEF15F0CA
:102A30000551095DD8A41FEF15F00451085DD8A019
:102A40002EEF15F0003F2EEF15F0013F2EEF15F0A1
:102A5000023F2EEF15F0032BD8B4120034B19EECD8
:102A600015F012000101346B9BEC15F0D8B0120088
:102A7000D0EC15F0200E366F0037013702370337E0
:102A800011EE33F00A0E376FE7360A0EE75CD8B066
:102A9000E76EE552372F44EF15F0362F3CEF15F077
:102AA00034B12981D890120001010A0E346F200E32
:102AB000366F11EE29F03451376F0A0ED890E65276
:102AC000D8B0E726E732372F5FEF15F00333023334
:102AD00001330033362F59EF15F0E750FF0FD8A020
:102AE0000335D8B0120029B19EEC15F01200045144
:102AF00000270551D8B0053D01270651D8B0063D45
:102B000002270751D8B0073D032712000051086F74
:102B10000151096F02510A6F03510B6F120001013D
:102B2000006B016B026B036B12000101046B056B00
:102B3000066B076B12000335D8A012000351800BFF
:102B4000001F011F021F031F003FAEEF15F0013FE2
:102B5000AEEF15F0023FAEEF15F0032B342B03253B
:102B600012000735D8A012000751800B041F051F63
:102B7000061F071F043FC4EF15F0053FC4EF15F013
:102B8000063FC4EF15F0072B342B07251200003742
:102B9000013702370337083709370A370B37120076
:102BA0000101296B2A6B2B6B2C6B2D6B2E6B2F6B02
:102BB000306B316B326B336B12002A510F0B2A6F63
:102BC0002B510F0B2B6F2C510F0B2C6F2D510F0B0B
:102BD0002D6F2E510F0B2E6F2F510F0B2F6F30516A
:102BE0000F0B306F31510F0B316F32510F0B326FB2
:082BF00033510F0B336F12008B
:10BF0000E844F926000C160C2B0C3F0C520C640C68
:10BF1000760C860C960CA50CB30CC10CCF0CDC0C6B
:06BF2000E80CF40C000C1B
:00000001FF
